:1000000012C0189518951895189518951895189563
:100010001895189518951895189518951895189578
:1000200018951895189504E00EBF0FE50DBF00E771
:1000300001BB0FE107BB10E0129512BB12950FE157
:1000400008BB0AD020E028BB07D023952A30D8F37C
:100050001395163088F3EFCF0F931F932F930091D2
:100060003F000F9304E618EC2DE12A95F1F71A955D
:10007000D9F70A95C1F70F9100933F002F911F9177
:040080000F9108953F
:00000001FF
